:020000040000FA
:0A0000000000000032EF00F04BD0CA
:080018009ED09EA8FED7AD6E3C
:1000200012000B6A0A6EFF0E0A260B2200D0D8A01F
:100030001200030E096EE60E02D8F5D7096AFE0F0C
:10004000086EE86A095AD8A012000000080600D01D
:10005000F8D7096A086E110EFF0F08360936FCE35F
:10006000086E1200006A4F0EAF6EB06A240EAC6EBE
:10007000900EAB6E00010F0EC16E070EB46E0FEE48
:100080007EF0ED6AE950EA10FCE1EF6AC69AC30E11
:10009000926EE00E936EC00E946E9280928270D03B
:1000A000F2A409D0F294104A112AD6CF0EF0D7CF7D
:1000B0000FF0817A11009EAA19D0060EAB1412E13E
:1000C000E2CF34F0E1CF33F0352A10EE5AF035505C
:1000D000E126000EE222AECFE7FF34C0E2FF33C0DC
:1000E000E1FF1100AE50AE50AB98AB881100355017
:1000F000365C14E0362AEACF09F0E9CF08F000EECA
:100100005AF03650E926000EEA22EF50326E09C04E
:10011000EAFF08C0E9FFD880120004D0E868326E18
:10012000D8A012001200356A366A9D8A9F8AF28E24
:10013000F28C12009D9A00EE5AF0010EF46EF36AF2
:10014000F306000EF45AEE6AF450F310F9E1356A42
:10015000366A9D8A1200F29EE0CF5AF4D8CF5BF443
:10016000E8CF5CF4F28E0001A192B36AB26AF29E0B
:100170005AC4E0FF5BC4D8FF5CC4E8FFF28E1000F5
:10018000939A8A8A0A0E4DDF939A8A9A9296899652
:1001900093948A94949A8B9A94988B9894968B962D
:1001A00094948B9494928B9294908B90929A899A37
:1001B00092988998226A00EE37F0200EEE68E82EB9
:1001C000FDD75780586A216AAEDFB4DFCD6AF2945A
:1001D000F28A870ED56EB16AA192A082B36AB26A22
:1001E000D08EA292B10EB16E25EC07F022EC0BF08E
:1001F000450E316E5780050E596ED6CF0EF0D7CF13
:100200000FF075DF32C012F0D90E125C07E3FE0E5C
:10021000125C01E301D0146A1CEF04F012AE38D076
:10022000146A880E125C05E112C014F01568166895
:100230002DD0980E125C05E112C014F017681868F2
:1002400025D0A80E125C05E112C014F019681A68D6
:100250001DD0B80E125C05E112C014F01B681C68BA
:1002600015D0C80E125C04E112C014F01D680ED047
:10027000D80E125C04E112C014F01E6807D0E80E1C
:10028000125C04E112C014F01F6820681BEF04F038
:10029000145204E11CEF04F01BEF04F0880E145C10
:1002A000D8A46FD0152803E112C015F066D012C093
:1002B00016F0160E155C0DE31550315C0AE3880E3E
:1002C000ACDE1550AADE1650A8DE585201E05806E2
:1002D00051D0155207E18B9A22903A6839683868F4
:1002E000376848D0010E155C07E18B9822923E6872
:1002F0003D683C683B683ED0020E155C07E18B967A
:1003000022944268416840683F6834D0030E155C0F
:1003100007E18B94229646684568446843682AD072
:10032000040E155C07E18B9222984A684968486878
:10033000476820D0050E155C07E18B90229A4E6825
:100340004D684C684B6816D0060E155C07E1899A1B
:10035000229C5268516850684F680CD0070E155C9B
:1003600007E18998229E566855685468536802D000
:100370001CEF04F015681BEF04F01CEF04F01BEFFA
:1003800004F0980E145CD8A4CAEF03F0172803E118
:1003900012C017F0FDD112C018F01852D8A462D0C4
:1003A000160E175C0DE31750315C0AE3980E35DE2C
:1003B000175033DE000E31DE585201E0580650D09F
:1003C000175207E18B9A22903A6839683868376883
:1003D00047D0010E175C07E18B9822923E683D687A
:1003E0003C683B683DD0020E175C07E18B96229477
:1003F0004268416840683F6833D0030E175C07E1EC
:100400008B942296466845684468436829D0040E58
:10041000175C07E18B9222984A68496848684768E8
:100420001FD0050E175C07E18B90229A4E684D682D
:100430004C684B6815D0060E175C07E1899A229C20
:100440005268516850684F680BD0070E175C07E17F
:100450008998229E566855685468536801D0ECD13B
:10046000EAD196D121A092D1160E175C0EE3175057
:10047000315C0BE3980E0DEC00F017500DEC00F022
:1004800018500DEC00F0582A81D117522DE118C0F8
:1004900024F08B8A7F0E245C21E2228003EE5AF046
:1004A000D8902434E926000EEA22EECF06F0EFCFF2
:1004B00007F006500E24026E07500F20036E000E48
:1004C0001020046E000E1120056E05C03AF004C025
:1004D00039F003C038F002C037F005D022903A68F6
:1004E00039683868376852D1010E175C2DE118C0A1
:1004F00025F08B887F0E255C21E2228203EE5AF0E4
:10050000D8902534E926000EEA22EECF06F0EFCF90
:1005100007F006500E24026E07500F20036E000EE7
:100520001020046E000E1120056E05C03EF004C0C0
:100530003DF003C03CF002C03BF005D022923E6883
:100540003D683C683B6822D1020E175C2DE118C063
:1005500026F08B867F0E265C21E2228403EE5AF081
:10056000D8902634E926000EEA22EECF06F0EFCF2F
:1005700007F006500E24026E07500F20036E000E87
:100580001020046E000E1120056E05C042F004C05C
:1005900041F003C040F002C03FF005D02294426811
:1005A000416840683F68F2D0030E175C2DE118C027
:1005B00027F08B847F0E275C21E2228603EE5AF01F
:1005C000D8902734E926000EEA22EECF06F0EFCFCE
:1005D00007F006500E24026E07500F20036E000E27
:1005E0001020046E000E1120056E05C046F004C0F8
:1005F00045F003C044F002C043F005D0229646689F
:10060000456844684368C2D0040E175C2DE118C0E9
:1006100028F08B827F0E285C21E2228803EE5AF0BC
:10062000D8902834E926000EEA22EECF06F0EFCF6C
:1006300007F006500E24026E07500F20036E000EC6
:100640001020046E000E1120056E05C04AF004C093
:1006500049F003C048F002C047F005D022984A682C
:1006600049684868476892D0050E175C2DE118C0AC
:1006700029F08B807F0E295C21E2228A03EE5AF05A
:10068000D8902934E926000EEA22EECF06F0EFCF0B
:1006900007F006500E24026E07500F20036E000E66
:1006A0001020046E000E1120056E05C04EF004C02F
:1006B0004DF003C04CF002C04BF005D0229A4E68BA
:1006C0004D684C684B6862D0060E175C2DE118C06F
:1006D0002AF0898A7F0E2A5C21E2228C03EE5AF0EE
:1006E000D8902A34E926000EEA22EECF06F0EFCFAA
:1006F00007F006500E24026E07500F20036E000E06
:100700001020046E000E1120056E05C052F004C0CA
:1007100051F003C050F002C04FF005D0229C526847
:10072000516850684F6832D0070E175C2DE118C031
:100730002BF089887F0E2B5C21E2228E03EE5AF08B
:10074000D8902B34E926000EEA22EECF06F0EFCF48
:1007500007F006500E24026E07500F20036E000EA5
:100760001020046E000E1120056E05C056F004C066
:1007700055F003C054F002C053F005D0229E5668D5
:1007800055685468536802D0176856D0176853D01C
:1007900053D051D0A80E145C0CE1192803E112C00B
:1007A00019F005D012C01AF062EC06F044D044D023
:1007B00042D0B80E145C14E11B2803E112C01BF0F8
:1007C0000DD012C01CF0B80E0DEC00F01B500DEC5B
:1007D00000F01C500DEC00F0B6EC06F02DD02BD044
:1007E000C80E145C10E11D280CE112C01DF0060EAD
:1007F0001D5C06E2C80E0DEC00F01D500DEC00F083
:100800001D681AD018D0D80E145C08E11E2804E127
:1008100012C01EF0ACEC06F00FD00DD0E80E145C48
:100820000AE11F2803E112C01FF004D012C020F01B
:10083000AAEC06F001D00CDA080E305CD8B080D1FA
:100840002C500E5C2D500F582E5010582F50115810
:10085000D8A068D12F8E30522AE122B006D08B9AD0
:100860003A6839683868376821D0827A949A03EEFA
:100870005AF0D8902434E926000EEA22EECF06F092
:10088000EFCF07F006500E24026E07500F20036EC4
:10089000000E1020046E000E1120056E05C03AF007
:1008A00004C039F003C038F002C037F03AD1010E6D
:1008B000305C2AE122B206D08B983E683D683C68E5
:1008C0003B6821D08278949803EE5AF0D890253472
:1008D000E926000EEA22EECF06F0EFCF07F0065031
:1008E0000E24026E07500F20036E000E1020046EBF
:1008F000000E1120056E05C03EF004C03DF003C09F
:100900003CF002C03BF00DD1020E305C2AE122B473
:1009100006D08B964268416840683F6821D0827655
:10092000949603EE5AF0D8902634E926000EEA2277
:10093000EECF06F0EFCF07F006500E24026E075000
:100940000F20036E000E1020046E000E1120056EA5
:1009500005C042F004C041F003C040F002C03FF0C7
:10096000E0D0030E305C2AE122B606D08B944668B4
:1009700045684468436821D08274949403EE5AF029
:10098000D8902734E926000EEA22EECF06F0EFCF0A
:1009900007F006500E24026E07500F20036E000E63
:1009A0001020046E000E1120056E05C046F004C034
:1009B00045F003C044F002C043F0B3D0040E305CF5
:1009C0002AE122B806D08B924A684968486847688D
:1009D00021D08272949203EE5AF0D8902834E926FE
:1009E000000EEA22EECF06F0EFCF07F006500E24FD
:1009F000026E07500F20036E000E1020046E000ED2
:100A00001120056E05C04AF004C049F003C048F04B
:100A100002C047F086D0050E305C2AE122BA06D02B
:100A20008B904E684D684C684B6821D082709490D2
:100A300003EE5AF0D8902934E926000EEA22EECFD0
:100A400006F0EFCF07F006500E24026E07500F207D
:100A5000036E000E1020046E000E1120056E05C0FE
:100A60004EF004C04DF003C04CF002C04BF059D022
:100A7000060E305C2AE122BC06D0899A5268516881
:100A800050684F6821D0807A929A03EE5AF0D8903D
:100A90002A34E926000EEA22EECF06F0EFCF07F067
:100AA00006500E24026E07500F20036E000E102019
:100AB000046E000E1120056E05C052F004C051F006
:100AC00003C050F002C04FF02CD0070E305C29E17B
:100AD00022BE06D08998566855685468536821D05C
:100AE0008078929803EE5AF0D8902B34E926000EC5
:100AF000EA22EECF06F0EFCF07F006500E24026E8A
:100B000007500F20036E000E1020046E000E1120FF
:100B1000056E05C056F004C055F003C054F002C085
:100B200053F096D811AE0BD0116A106A0F6A0E6A94
:100B3000226A00EE37F0200EEE68E82EFDD706D0D0
:100B400011AE04D0116A106A0F6A0E6A0F5057185E
:100B5000020BD8A47AD0577257A077D0010E595CF7
:100B600006E1585202E08B8401D08B946ED0020EC5
:100B7000595C06E1585202E08B8601D08B9665D015
:100B8000030E595C08E1585203E08B8A8B8802D02F
:100B90008B9A8B985AD0040E595C0DE1585208E09C
:100BA00057B203D08B9A8B8802D08B8A8B9802D055
:100BB0008B9A8B984AD0050E595C20E1585029EC4D
:100BC00000F0136E135205E18B948B968B9A8B98E1
:100BD00014D0010E135C05E18B848B968B9A8B9855
:100BE0000CD0020E135C05E18B848B8A8B888B986A
:100BF00004D08B848B8A8B888B8627D0060E595C19
:100C000011E158B0828658A0829658B2828458A2C8
:100C1000829458B4828A58A4829A58B4828858A47C
:100C2000829813D0070E595C10E158B0828458A006
:100C3000829458B2828658A2829658B4828A58A466
:100C4000829A58B4828858A482988170FDEF00F08F
:100C500030682F8E136A080E135C33E2D890133479
:100C6000E96EEA6AEA36E936EA36370EE926000E18
:100C7000EA22EFCF02F0ECCF03F0ECCF04F0ECCFA0
:100C800005F02C50025C2D5003582E5004582F5064
:100C9000055815E2D8901334E96EEA6AEA36E93667
:100CA000EA36370EE926000EEA22EFCF2CF0ECCF21
:100CB0002DF0ECCF2EF0ECCF2FF013C030F0132A34
:100CC000CAE31200160E195C0DE31950315C0AE3F9
:100CD000A80E0DEC00F019500DEC00F01A500DECC0
:100CE00000F02ED0195203E11AC024F029D0010ED1
:100CF000195C03E11AC025F023D0020E195C03E150
:100D00001AC026F01DD0030E195C03E11AC027F0AB
:100D100017D0040E195C03E11AC028F011D0050E9B
:100D2000195C03E11AC029F00BD0060E195C03E12F
:100D30001AC02AF005D0070E195C02E11AC02BF088
:100D400019681200C80E0DEC00F01D500DEC00F0FB
:100D50001D6812001F681200585206E0D80E0DECF4
:100D600000F01E500DEC00F01E6812001E0E1B5C01
:100D700011E11CC024F01CC025F01CC026F01CC0D2
:100D800027F01CC028F01CC029F01CC02AF01CC091
:100D90002BF03ED0420E1B5C09E11C5203E1219076
:100DA00039D803D089868A84218032D0450E1B5CD5
:100DB00012E11C5202E0578006D05790586A8B9A75
:100DC0008B988B968B941CC059F0080E595C02E3EB
:100DD000070E596E1DD05A0E1B5C0DE11CC031F080
:100DE000160E315C02E2160E316E460E315C02E3E5
:100DF000450E316E0DD07B0E1B5C0AE1226A8B9A88
:100E00008B988B968B948B928B90899A8998586A41
:100E10001B68120089968A94226A246A256A266AC7
:100E2000276A286A296A2A6A2B6A8B9A8B988B967A
:100E30008B948B928B90899A8998216A450E316E9A
:100E4000586A5780050E596E120002015B695A6993
:100E50005C0E5D6F7A0E5C6F590E5F6F850E5E6F74
:100E6000580E616F140E606F560E636FA90E626F9D
:100E7000550E656F430E646F530E676FE30E666F1A
:100E8000520E696F890E686F510E6B6F350E6A6F67
:100E90004F0E6D6FE60E6C6F4E0E6F6F9C0E6E6F89
:100EA0004D0E716F580E706F4C0E736F190E726F7E
:100EB0004A0E756FDF0E746F490E776FAA0E766F4C
:100EC000480E796F7A0E786F470E7B6F4F0E7A6FF0
:100ED000460E7D6F290E7C6F450E7F6F080E7E6F6C
:100EE000430E816FEB0E806F420E836FD30E826FC5
:100EF000410E856FBF0E846F400E876FB00E866FF8
:100F00003F0E896FA50E886F3E0E8B6F9E0E8A6F07
:100F10003D0E8D6F9C0E8C6F3C0E8F6F9E0E8E6FF4
:100F20003B0E916FA40E906F3A0E936FAE0E926FC0
:100F3000390E956FBC0E946F380E976FCE0E966F6C
:100F4000370E996FE30E986F360E9B6FFD0E9A6FFA
:100F5000360E9D6F1A0E9C6F350E9F6F3B0E9E6F67
:100F6000340EA16F5F0EA06F330EA36F870EA26FBA
:100F7000320EA56FB20EA46F310EA76FE10EA66FF1
:100F8000310EA96F140EA86F300EAB6F490EAA6F09
:100F90002F0EAD6F820EAC6F2E0EAF6FBE0EAE6F0A
:100FA0002D0EB16FFD0EB06F2D0EB36F3F0EB26FF1
:100FB0002C0EB56F850EB46F2B0EB76FCD0EB66FBE
:100FC0002B0EB96F180EB86F2A0EBB6F670EBA6F73
:100FD000290EBD6FB80EBC6F290EBF6F0C0EBE6F11
:100FE000280EC16F620EC06F270EC36FBC0EC26F9A
:100FF000270EC56F180EC46F260EC76F760EC66F0C
:10100000250EC96FD80EC86F250ECB6F3C0ECA6F68
:10101000240ECD6FA20ECC6F240ECF6F0B0ECE6FB1
:10102000230ED16F760ED06F220ED36FE40ED26FE7
:10103000220ED56F540ED46F210ED76FC60ED66F09
:10104000210ED96F3B0ED86F200EDB6FB20EDA6F18
:10105000200EDD6F2B0EDC6F1F0EDF6FA60EDE6F16
:101060001F0EE16F240EE06F1E0EE36FA30EE26F02
:101070001E0EE56F250EE46F1D0EE76FA90EE66FDD
:101080001D0EE96F2E0EE86F1C0EEB6FB60EEA6FA9
:101090001C0EED6F3F0EEC6F1B0EEF6FCB0EEE6F65
:1010A0001B0EF16F580EF06F1A0EF36FE80EF26F11
:1010B0001A0EF56F790EF46F1A0EF76F0B0EF66FAE
:1010C000190EF96FA00EF86F190EFB6F360EFA6F3E
:1010D000180EFD6FCE0EFC6F180EFF6F680EFE6FC0
:1010E000180E0301016F030E006F170E036FA00EA1
:1010F000026F170E056F3F0E046F160E076FDF0E9F
:10110000066F160E096F800E086F160E0B6F240EF9
:101110000A6F150E0D6FC80E0C6F150E0F6F6E0E49
:101120000E6F150E116F160E106F140E136FBF0E8B
:10113000126F140E156F690E146F140E176F150EC3
:10114000166F130E196FC20E186F130E1B6F710EF0
:101150001A6F130E1D6F210E1C6F120E1F6FD20E11
:101160001E6F120E216F840E206F120E236F380E29
:10117000226F110E256FED0E246F110E276FA30E37
:10118000266F110E296F5A0E286F110E2B6F120E3B
:101190002A6F100E2D6FCC0E2C6F100E2F6F870E36
:1011A0002E6F100E316F420E306F0F0E336F32699B
:1011B000356FBD0E346F0F0E376F7C0E366F0F0E0E
:1011C000396F3D0E386F0E0E3B6FFE0E3A6F0E0EEE
:1011D0003D6FC00E3C6F0E0E3F6F830E3E6F0E0EC6
:1011E000416F470E406F0E0E436F0C0E426F0D0E97
:1011F000456FD20E446F0D0E476F990E466F0D0E60
:10120000496F610E486F0D0E4B6F2A0E4A6F0C0E20
:101210004D6FF40E4C6F0C0E4F6FBE0E4E6F0C0EDA
:10122000516F8A0E506F0C0E536F560E526F0C0E8C
:10123000556F230E546F0B0E576FF10E566F0B0E3A
:10124000596FC00E586F5B695A69A20E5D6FC30E6D
:101250005C6F9A0E5F6F460E5E6F960E616F320E78
:10126000606F920E636F3A0E626F8E0E656F5D0E49
:10127000646F8A0E676F9A0E666F860E696FF00E46
:10128000686F830E6B6F5F0E6A6F7F0E6D6FE70E78
:101290006C6F7C0E6F6F850E6E6F790E716F3B0EEB
:1012A000706F760E736F070E726F720E756FE80EA9
:1012B000746F6F0E776FDF0E766F6C0E796FEA0EBC
:1012C000786F6A0E7B6F0A0E7A6F670E7D6F3C0E29
:1012D0007C6F640E7F6F820E7E6F610E816FDA0EFF
:1012E000806F5F0E836F440E826F5C0E856FBF0E42
:1012F000846F5A0E876F4C0E866F570E896FE90EFA
:10130000886F550E8B6F960E8A6F530E8D6F8C6F94
:10131000510E8F6F200E8E6F4E0E916FFB0E906FE1
:101320004C0E936FE50E926F4A0E956FDC0E946F24
:10133000480E976FE20E966F460E996FF50E986FF6
:10134000450E9B6F150E9A6F430E9D6F420E9C6F5C
:10135000410E9F6F7B0E9E6F3F0EA16FC00EA06F60
:101360003E0EA36F100EA26F3C0EA56F6D0EA46F04
:101370003A0EA76FD40EA66F390EA96F460EA86F4E
:10138000370EAB6FC20EAA6F360EAD6F490EAC6F43
:10139000340EAF6FDA0EAE6F330EB16F740EB06FE6
:1013A000320EB36F180EB26F300EB56FC50EB46F3C
:1013B0002F0EB76F7B0EB66F2E0EB96F3A0EB86F49
:1013C0002D0EBB6F020EBA6F2B0EBD6FD10EBC6F10
:1013D0002A0EBF6FA90EBE6F290EC16F880EC06F97
:1013E000280EC36F6F0EC26F270EC56F5E0EC46FDF
:1013F000260EC76F530EC66F250EC96F500EC86FED
:10140000240ECB6F540ECA6F230ECD6F5E0ECC6FC1
:10141000220ECF6F6F0ECE6F210ED16F860ED06F62
:10142000200ED36FA30ED26F1F0ED56FC60ED46FD2
:101430001E0ED76FEF0ED66F1E0ED96FD86F1D0E12
:10144000DB6F520EDA6F1C0EDD6F8C0EDC6F1B0E25
:10145000DF6FCB0EDE6F1B0EE16F0F0EE06F1A0E0B
:10146000E36F580EE26F190EE56FA50EE46F180ECC
:10147000E76FF80EE66F180EE96F4F0EE86F170E64
:10148000EB6FAB0EEA6F170EED6F0A0EEC6F160ED8
:10149000EF6F6F0EEE6F150EF16FD70EF06F150E2A
:1014A000F36F430EF26F140EF56FB30EF46F140E5C
:1014B000F76F270EF66F130EF96F9F0EF86F130E6E
:1014C000FB6F1A0EFA6F120EFD6F990EFC6F120E63
:1014D000FF6F1B0EFE6F110E0401016FA10E006F56
:1014E000110E036F290E026F100E056FB50E046FFB
:1014F000100E076F440E066F0F0E096FD60E086FA1
:101500000F0E0B6F6B0E0A6F0F0E0D6F030E0C6F2D
:101510000E0E0F6F9D0E0E6F0E0E116F3A0E106FA6
:101520000D0E136FDA0E126F0D0E156F7C0E146F09
:101530000D0E176F210E166F0C0E196FC80E186F57
:101540000C0E1B6F720E1A6F0C0E1D6F1E0E1C6F91
:101550000B0E1F6FCC0E1E6F0B0E216F7C0E206FBB
:101560000B0E236F2E0E226F0A0E256FE30E246FD3
:101570000A0E276F990E266F0A0E296F510E286FDB
:101580000A0E2B6F0B0E2A6F090E2D6FC80E2C6FD3
:10159000090E2F6F850E2E6F090E316F450E306FBD
:1015A000090E336F060E326F080E356FC90E346F99
:1015B000080E376F8E0E366F080E396F540E386F67
:1015C000080E3B6F1C0E3A6F070E3D6FE50E3C6F29
:1015D000070E3F6FAF0E3E6F070E416F7B0E406FE1
:1015E000070E436F490E426F070E456F170E446F8B
:1015F000060E476FE70E466F060E496FB90E486F2D
:10160000060E4B6F8B0E4A6F060E4D6F5F0E4C6FC2
:10161000060E4F6F340E4E6F060E516F0A0E506F4E
:10162000050E536FE10E526F050E556FB90E546FD4
:10163000050E576F930E566F050E596F6D0E586F4E
:1016400000011200040E01015D6F880E5C6F040E34
:101650005F6FA60E5E6F040E616FB60E606F040EB4
:10166000636FC60E626F040E656FD60E646F040E54
:10167000676FE60E666F040E696FF60E686F050EF3
:101680006B6F070E6A6F050E6D6F170E6C6F050E90
:101690006F6F280E6E6F050E716F390E706F050E2D
:1016A000736F4B0E726F050E756F5D0E746F050EC6
:1016B000776F6E0E766F050E796F800E786F050E60
:1016C0007B6F930E7A6F050E7D6FA50E7C6F050EF6
:1016D0007F6FB80E7E6F050E816FCB0E806F050E8B
:1016E000836FDF0E826F050E856FF20E846F060E1C
:1016F000876F866F896F1A0E886F060E8B6F2E0E9E
:101700008A6F060E8D6F430E8C6F060E8F6F580E0C
:101710008E6F060E916F6D0E906F060E936F830E97
:10172000926F060E956F980E946F060E976FAE0E21
:10173000966F060E996FC40E986F060E9B6FDB0EA8
:101740009A6F060E9D6FF20E9C6F070E9F6F090E2B
:101750009E6F070EA16F210EA06F070EA36F380EAC
:10176000A26F070EA56F500EA46F070EA76F690E2C
:10177000A66F070EA96F810EA86F070EAB6F9A0EAA
:10178000AA6F070EAD6FB40EAC6F070EAF6FCD0E24
:10179000AE6F070EB16FE70EB06F080EB36F020E9B
:1017A000B26F080EB56F1D0EB46F080EB76F380E0E
:1017B000B66F080EB96F530EB86F080EBB6F6F0E81
:1017C000BA6F080EBD6F8B0EBC6F080EBF6FA70EF1
:1017D000BE6F080EC16FC40EC06F080EC36FE10E5E
:1017E000C26F080EC56FC469090EC76F1D0EC66FA4
:1017F000090EC96F3B0EC86F090ECB6F5A0ECA6F28
:10180000090ECD6F790ECC6F090ECF6F990ECE6F8A
:10181000090ED16FB90ED06F090ED36FD90ED26FEA
:10182000090ED56FFA0ED46F0A0ED76F1B0ED66F46
:101830000A0ED96F3D0ED86F0A0EDB6F5F0EDA6F9E
:101840000A0EDD6F820EDC6F0A0EDF6FA50EDE6FF3
:101850000A0EE16FC80EE06F0A0EE36FEC0EE26F46
:101860000B0EE56F110EE46F0B0EE76F360EE66F91
:101870000B0EE96F5B0EE86F0B0EEB6F810EEA6FDC
:101880000B0EED6FA70EEC6F0B0EEF6FCE0EEE6F23
:101890000B0EF16FF50EF06F0C0EF36F1D0EF26F65
:1018A0000C0EF56F460EF46F0C0EF76F6F0EF66FA1
:1018B0000C0EF96F980EF86F0C0EFB6FC20EFA6FDC
:1018C0000C0EFD6FED0EFC6F0D0EFF6F180EFE6F10
:1018D0000D0E0201016F430E006F0D0E036F700EAF
:1018E000026F0D0E056F9C0E046F0D0E076FCA0E72
:1018F000066F0D0E096FF80E086F0E0E0B6F260E99
:101900000A6F0E0E0D6F550E0C6F0E0E0F6F850EBB
:101910000E6F0E0E116FB60E106F0E0E136FE70ED8
:10192000126F0F0E156F180E146F0F0E176F4B0EF0
:10193000166F0F0E196F7E0E186F0F0E1B6FB10E04
:101940001A6F0F0E1D6FE60E1C6F100E1F6F1B0E11
:101950001E6F100E216F500E206F100E236F870E1A
:10196000226F100E256FBE0E246F100E276FF60E1D
:10197000266F110E296F2E0E286F110E2B6F680E19
:101980002A6F110E2D6FA20E2C6F110E2F6FDC0E11
:101990002E6F120E316F180E306F120E336F540E01
:1019A000326F120E356F910E346F120E376FCF0EED
:1019B000366F130E396F0E0E386F130E3B6F4D0ED0
:1019C0003A6F130E3D6F8E0E3C6F130E3F6FCF0EAE
:1019D0003E6F140E416F110E406F140E436F540E84
:1019E000426F140E456F980E446F140E476FDC0E55
:1019F000466F150E496F220E486F150E4B6F680E1D
:101A00004A6F150E4D6FB00E4C6F150E4F6FF80EDE
:101A10004E6F160E516F410E506F160E536F8C0E97
:101A2000526F160E556FD70E546F170E576F230E49
:101A3000566F170E596F700E586F00011200FFD7C6
:020000040030CA
:0300010006160ED2
:020005008580F4
:060008000FC00FE00F40E5
:00000001FF
